:1000000038C052C051C050C04FC04EC04DC04CC08F
:100010004BC0F8C049C048C047C046C045C044C0F6
:1000200043C042C041C0000037343100003835328F
:100030000000363330040404040404040402020201
:100040000202020303030303030102040810204019
:1000500080010204081020010204081020000000A2
:100060000000000000000304050000000000000084
:10007000000011241FBECFE5D4E0DEBFCDBF10E0ED
:10008000A0E6B0E0E0E0F5E002C005900D92A037F8
:10009000B107D9F710E0A0E7B0E001C01D92A83782
:1000A000B107E1F7ABD02BC2ABCF10927300109227
:1000B000720060E070E080916A0047D16FEF70E0FD
:1000C0008091720090917300681B790B80916E0093
:1000D0003CD16EE170E080E090E0D0D060917200A1
:1000E000709173006B5F7F4F709373006093720029
:1000F0006F3F710501F3FCF21092730010927200D1
:1001000060E070E080916E0020D16FEF70E0809130
:10011000720090917300681B790B80916C0015D16F
:100120006EE170E080E090E0A9D060917200709183
:1001300073006B5F7F4F70937300609372006F3F2B
:10014000710501F3FCF2109273001092720060E0EE
:1001500070E080916C00F9D06FEF70E080917200D8
:1001600090917300681B790B80916A00EED06EE16C
:1001700070E080E090E082D0609172007091730036
:100180006B5F7F4F70937300609372006F3F7105D8
:1001900001F3FCF2089560E08091600005D160E019
:1001A0008091620001D160E080916400FDD060E048
:1001B00080916600F9D061E080916800F5D061E03F
:1001C00080916A00F1D061E080916C00EDD061E037
:1001D00080916E00E9D061E08091680039D16AE0D9
:1001E00070E080E090E04AD060E08091680030D11B
:1001F0002ED0709371006093700008956CD0CBDFA7
:1002000054DFFECF1F920F920FB60F9211248F93DF
:100210009F93AF93BF938091740090917500A091CC
:100220007600B09177000196A11DB11D80937400F6
:1002300090937500A0937600B0937700BF91AF9133
:100240009F918F910F900FBE0F901F901895609106
:10025000740070917500809176009091770027E08E
:10026000660F771F881F991F2A95D1F72DE730E079
:1002700040E050E022D1CA01B9010895AF92BF9287
:10028000CF92DF92EF92FF920F931F935B016C016D
:10029000DEDF7B018C01DBDF6E197F09800B910BA8
:1002A0006A157B058C059D05B0F31F910F91FF909A
:1002B000EF90DF90CF90BF90AF900895019751F0ED
:1002C000880F991F880F991F02972FB7F8940197ED
:1002D000F1F72FBF08957894109274001092750072
:1002E000109276001092770083B7826083BF83B745
:1002F000816083BF89B7816089BF8EB582608EBD02
:100300008EB581608EBD8FB581608FBD85B58460EF
:1003100085BD85B5806485BD3F983E9A329A319AF5
:10032000309A379A1AB8089597B1907F8F70982BAA
:1003300097B9369A3699FECF24B185B19927982F6F
:1003400088273327822B932B08951F93CF93DF9316
:10035000182FEB0161E028D0E12FFF27E35AFF4F70
:100360008491833031F48FB580688FBDDBBDCABD09
:1003700017C0843031F48FB580628FBDD9BDC8BD40
:100380000FC0853029F485B5806285BDC3BD08C026
:10039000C038D10514F460E001C061E0812F58D06D
:1003A000DF91CF911F910895282F3327C901875BD3
:1003B0009F4FFC0194912B5C3F4FF901849188235E
:1003C00081F0E82FFF27EA5DFF4FE491FF276623C6
:1003D00029F4808190958923808308958081892BD9
:1003E00080830895482F5527CA01835A9F4FFC01E7
:1003F0002491CA01875B9F4FFC0194914B5C5F4F36
:10040000FA013491332319F480E090E00895222317
:1004100081F0233019F48FB58F7704C0243021F494
:100420008FB58F7D8FBD05C0253019F485B58F7DC3
:1004300085BDE32FFF27E05DFF4FE491FF2780811B
:1004400020E030E0892311F021E030E0C901089577
:10045000482F5527CA01835A9F4FFC012491CA0196
:10046000875B9F4FFC0194914B5C5F4FFA01349185
:10047000332311F1222381F0233019F48FB58F77C4
:1004800004C0243021F48FB58F7D8FBD05C0253089
:1004900019F485B58F7D85BDE32FFF27E55DFF4FFF
:1004A000E491FF27662329F4808190958923808336
:1004B00008958081892B80830895A1E21A2EAA1BBA
:1004C000BB1BFD010DC0AA1FBB1FEE1FFF1FA21704
:1004D000B307E407F50720F0A21BB30BE40BF50B01
:1004E000661F771F881F991F1A9469F7609570958A
:1004F000809590959B01AC01BD01CF010895FFCF80
:100500000200030004000500060009000A000B00B9
:00000001FF
